:1000000026C03EC03DC03CC03BC01AC139C038C04C
:1000100037C036C035C034C033C032C031C0000034
:10002000000037000000000038000000000036002B
:10003000020202020202020202020102040810206D
:100040002004100801020000040000000000112438
:100050001FBECFEDCDBF10E0A0E6B0E0E8EAF5E0CE
:1000600002C005900D92A236B107D9F720E0A2E6B2
:10007000B0E001C01D92A937B207E1F72BD192C2BF
:10008000BFCF823081F018F4813051F00895833071
:1000900019F0843009F008958CB58F7D8CBD0895DA
:1000A0008AB58F7702C08AB58F7D8ABD08951F9368
:1000B000CF93DF93282F30E0F901EC5BFF4F849161
:1000C000F901E65CFF4FD491F901E05DFF4FC49167
:1000D000CC23C1F0162F8111D4DFEC2FF0E0EE0F0E
:1000E000FF1FEC5DFF4FA591B4918FB7F8941111EC
:1000F00005C09C91ED2FE095E92302C0EC91ED2B1A
:10010000EC938FBFDF91CF911F910895CF93DF9331
:1001100090E0FC01E65CFF4F2491FC01E05DFF4FA5
:100120008491882361F190E0880F991FFC01E25EC1
:10013000FF4FC591D491FC01EC5DFF4FA591B491A7
:10014000611109C09FB7F894888120958223888324
:10015000EC912E230BC0623061F49FB7F894388184
:10016000822F809583238883EC912E2B2C939FBF25
:1001700006C08FB7F894E8812E2B28838FBFDF91BC
:10018000CF9108953FB7F8948091630090916400F7
:10019000A0916500B091660022B708B601FE05C0C7
:1001A0002F3F19F00196A11DB11D3FBFBA2FA92FF6
:1001B000982F8827820F911DA11DB11DBC01CD0173
:1001C00042E0660F771F881F991F4A95D1F708955F
:1001D0008F929F92AF92BF92CF92DF92EF92FF9257
:1001E0006B017C01CFDF4B015C01C114D104E10440
:1001F000F104E9F0C7DFDC01CB0188199909AA09EC
:10020000BB09883E9340A105B10578F321E0C21AED
:10021000D108E108F10888EE880E83E0981EA11C41
:10022000B11CC114D104E104F10421F7DECFFF9029
:10023000EF90DF90CF90BF90AF909F908F900895F8
:100240001F920F920FB60F9211242F933F938F930B
:100250009F93AF93BF938091670090916800A091A6
:100260006900B0916A003091620023E0230F2D37BE
:1002700020F40196A11DB11D05C026E8230F0296AA
:10028000A11DB11D209362008093670090936800C8
:10029000A0936900B0936A0080916300909164001C
:1002A000A0916500B09166000196A11DB11D8093DB
:1002B000630090936400A0936500B0936600BF91C3
:1002C000AF919F918F913F912F910F900FBE0F9003
:1002D0001F90189578948AB582608ABD8AB581602E
:1002E0008ABD83B7826083BF83B7816083BF89B7CC
:1002F000826089BF80B7826080BF80B7816080BF25
:10030000329A319A309A379A8CB580648CBD61E00C
:1003100081E0FCDE61E080E0F9DE60E083E0F6DEB3
:1003200060E081E0C4DE60E080E0C1DE1092780031
:100330001092770010926C0010926B00C7E4D0E02E
:100340000DE310E033E3E32E30E0F32E45E4C42E5A
:1003500040E0D42EAA24AA94B12C20E0822E20E0E2
:10036000922E61E081E0A3DEFE018491F8016490A9
:10037000F7017490772089F0811183DEE72DF0E09A
:10038000EE0FFF1FE65DFF4FA591B4918C9168229F
:1003900091E080E021F490E002C090E080E0909352
:1003A0007700809378002FB7F89480916700909140
:1003B0006800A0916900B0916A002FBF809373001C
:1003C00090937400A0937500B09376008054984D7C
:1003D000A64FBF4F80936F0090937000A093710061
:1003E000B09372008091770090917800019709F0A6
:1003F00058C061E080E05BDE54C02FB7F8944091B4
:100400006700509168006091690070916A002FBF89
:10041000409373005093740060937500709376005E
:1004200040906F005090700060907100709072006A
:10043000441655066606770608F474C060906D0091
:1004400070906E0061E081E061DE6114710491F5ED
:1004500060E081E02CDE20916000309161008091AD
:100460006D0090916E00820F931F90936E008093A9
:100470006D00AC01415051094E3F510508F044C098
:1004800080916D0090916E008F3F910529F024F0CE
:10049000B0926E00A0926D0064E170E080E090E0A8
:1004A00097DE80917700909178008130910509F472
:1004B000A4CF41C0FFEF6F16710411F461E0C9CF02
:1004C000F6018491823089F038F48130C1F48AB524
:1004D00080688ABD69BCBFCF833061F0843079F415
:1004E0008CB580628CBD6BBCB6CF8AB580628ABD8C
:1004F00068BCB1CF8CB580628CBD6EBCACCFF0E86F
:100500006F167104DCF6A4CF319521953109309333
:1005100061002093600097FFB3CF10926E0010929D
:100520006D00AECF109278001092770090936C001F
:1005300080936B00B1CF60E081E0B9DD60E080E0E6
:10054000B6DD80916B0090916C00019771F0109274
:100550006C0010926B00109278001092770081145A
:10056000910409F4FECE4CDDF8CE85E0682E712CA6
:1005700062E370E080E090E02BDE61E081E097DDF7
:1005800064E670E080E090E023DE60E081E08FDDF3
:1005900064E670E080E090E01BDE81E0681A71089C
:0805A00039F7D5CFF894FFCF25
:0205A800080049
:00000001FF
